:0200000480007A
:100000006F000005732F2034930F80006308FF03F7
:10001000930F90006304FF03930FB0006300FF038E
:10002000130F000063040F0067000F00732F2034CC
:1000300063540F006F00400093E19153171F0000BD
:1000400023223FFC171F000023200FFC6FF01FFF2F
:100050009300000013010000930100001302000050
:100060009302000013030000930300001304000038
:100070009304000013050000930500001306000020
:100080009306000013070000930700001308000008
:10009000930800001309000093090000130A0000F0
:1000A000930A0000130B0000930B0000130C0000D8
:1000B000930C0000130D0000930D0000130E0000C0
:1000C000930E0000130F0000930F0000732540F102
:1000D0006310050097020000938202017390523072
:1000E000735044749702000093820201739052305F
:1000F00073500018970200009382420273905230AE
:100100009B021000939252039382F2FF7390023B82
:100110009302F0017390023A73504030970200004E
:1001200093824201739052307350203073503030BC
:100130009301000097020000938202ED7390523009
:10014000130510001315F501635C05000F00F00F97
:10015000930110009308D005130500007300000000
:1001600093020000638A020073905210B7B200003D
:100170009B829210739022307350003097020000DF
:100180009382420173901234732540F17300203042
:100190009301200093001000130100003B97200002
:1001A00093031000631C775E9301300093001000EE
:1001B000130110003B972000930320006310775E2B
:1001C0009301400093001000130170003B97200042
:1001D000930300086314775C9301500093001000B0
:1001E0001301E0003B972000B74300006318775AE3
:1001F00093016000930010001301F0013B97200071
:10020000B7030080631C7758930170009300F0FFE0
:10021000130100003B9720009303F0FF6310775811
:10022000930180009300F0FF130110003B97200022
:100230009303E0FF63147756930190009300F0FF5F
:10024000130170003B972000930300F86318775464
:100250009301A0009300F0FF1301E0003B97200002
:10026000B7C3FFFF631C77529301B0009300F0FF08
:100270001301F0013B972000B70300806310775211
:100280009301C000B72021219B80101213010000B0
:100290003B972000B72321219B83131263107750D3
:1002A0009301D000B72021219B8010121301100070
:1002B0003B972000B74342429B8323246310774E31
:1002C0009301E000B72021219B80101213017000E0
:1002D0003B972000B79390909B8303086310774C63
:1002E0009301F000B72021219B8010121301E00040
:1002F0003B972000B74348486312774A93010001B7
:10030000B72021219B8010121301F0013B972000A0
:10031000B70300806314774893011001B7202121AF
:100320009B801012130100FE3B972000B723212170
:100330009B8313126314774693012001B720212178
:100340009B801012130110FE3B972000B7434242DE
:100350009B8323246314774493013001B720212128
:100360009B801012130170FE3B972000B793909072
:100370009B8303086314774293014001B720212136
:100380009B8010121301E0FE3B972000B7434848C2
:100390006316774093015001B72021219B801012F2
:1003A0001301F0FF3B972000B70300806318773EEE
:1003B0009301C002B720F1FF9B8050349390C0009E
:1003C00093808067130100003B972000B7533412DD
:1003D0009B8383676314773C9301D002B720F1FFBE
:1003E0009B8050349390C00093808067130140003D
:1003F0003B972000B76345239B8303786310773ACC
:100400009301E002B72009009B8050349390C00014
:1004100093808067130100003B972000B75334920C
:100420009B838367631C77369301F002B7900900C2
:100430009B8050349390C0009380806713014000EC
:100440003B972000B76345939B8303786318773409
:10045000930160019300100013017000BB90200015
:1004600093030008639C70329301700193001000A5
:100470001301E0003B912000B7430000631071328C
:100480009301800193003000BB9010009303800122
:1004900063967030930190011302000093001000E6
:1004A000130170003B972000130307001302120092
:1004B00093022000E31452FE930300086310732E8E
:1004C0009301A00113020000930010001301E0004B
:1004D0003B972000130000001303070013021200D3
:1004E00093022000E31252FEB74300006318732A00
:1004F0009301B00113020000930010001301F001FA
:100500003B972000130000001300000013030700B6
:100510001302120093022000E31052FEB703008082
:10052000631E73269301C0011302000093001000A4
:10053000130170003B972000130212009302200069
:10054000E31652FE93030008631A77249301D00147
:1005500013020000930010001301E00013000000DC
:100560003B9720001302120093022000E31452FE76
:10057000B7430000631477229301E00113020000E7
:10058000930010001301F00113000000130000009D
:100590003B9720001302120093022000E31252FE48
:1005A000B7030080631C771E9301F0011302000063
:1005B0009300100013000000130170003B9720000F
:1005C0001302120093022000E31452FE930300086A
:1005D0006316771C930100021302000093001000C1
:1005E000130000001301E000130000003B972000FF
:1005F0001302120093022000E31252FEB7430000E0
:10060000631E77189301100213020000930010007C
:1006100013000000130000001301F0013B972000BD
:100620001302120093022000E31252FEB70300806F
:100630006316771693012002130200001301700065
:10064000930010003B972000130212009302200039
:10065000E31652FE930300086312771493013002ED
:10066000130200001301E0009300100013000000CB
:100670003B9720001302120093022000E31452FE65
:10068000B7430000631C771093014002130200007F
:100690001301F0019300100013000000130000008C
:1006A0003B9720001302120093022000E31252FE37
:1006B000B70300806314770E930150021302000009
:1006C0001301700013000000930010003B972000FE
:1006D0001302120093022000E31452FE9303000859
:1006E000631E770A93016002130200001301E00009
:1006F0001300000093001000130000003B9720003F
:100700001302120093022000E31252FEB7430000CE
:100710006316770893017002130200001301F001C1
:100720001300000013000000930010003B9720000E
:100730001302120093022000E31252FEB70300805E
:10074000631E7704930180029300F0003B111000B8
:10075000930300006314710493019002930000025C
:100760003B91000093030002631A71029301A002FF
:10077000BB10000093030000639270029301B0026B
:1007800093000040371100001B0101803B902000C6
:100790009303000063147000631030020F00F00F29
:1007A000638001009391110093E111009308D0053B
:1007B00013850100730000000F00F00F930110007B
:1007C0009308D0051305000073000000731000C0EB
:1007D0000000000000000000000000000000000019
:1007E0000000000000000000000000000000000009
:0C07F000000000000000000000000000FD
:1010000000000000000000000000000000000000E0
:1010100000000000000000000000000000000000D0
:1010200000000000000000000000000000000000C0
:1010300000000000000000000000000000000000B0
:081040000000000000000000A8
:040000058000000077
:00000001FF
